:100000000C941E060C94BC270C94E9270C9446060D
:100010000C9446060C94DC120C9446060C9446068E
:100020000C9446060C9446060C9446060C94460620
:100030000C9446060C9446060C9446060C94460610
:100040000C9416280C9446060C94042C0C94472C03
:100050000C9446060C9446060C9446060C944606F0
:100060000C9446060C9446064618A81887188A1859
:100070008D189018931896189918A818A218DA19BC
:10008000DC19DC19DA19DC19DC19DC19DC19DC19CA
:10009000DC19DC19DC19DC19DC19DC19DC19DC19B8
:1000A0006019DC19DC19DC19DC19DC19D118DC1930
:1000B000DC19DC19DC19DC19DC19DC19DC19DC1998
:1000C000DC19DC19DC19DC19DC19DC196C196C1968
:1000D0006C196C196C196C196C196C196C19DC1988
:1000E000DC19DC19DC19DC19DC19D1186B196B1956
:1000F0006B196B19DC1979197F1985198B199119ED
:1001000097199D19A319AD19B719C119CB1912194E
:10011000D418DC19DC19DC19DC196019DC19DC19BC
:10012000DC19DC19DC19DC19DC19DC196A196A190B
:100130006A196A19DC1979197F1985198B199119AE
:1001400097199D19A319AD19B719C119CB1912190E
:10015000D418DC19DC19DC19DC1960190F1A0F1A14
:100160000F1A0F1A0F1A0F1A0F1A0F1A0F1A0F1A47
:100170000F1A0F1A0F1A261B261B261B261B261BBF
:10018000261B541A5E1A681A721AD01ADA1AE91A59
:10019000FA1A821C971CA31CAC1CBB1CE01CE91C9B
:1001A000321DFB1C45204B20512058206620882002
:1001B000A620456E746572206D656E752E2E2E001C
:1001C000546F67676C6564206D6963726F50504D42
:1001D00000546F67676C656420696E76657274653C
:1001E000642050504D2100546F67676C6564205443
:1001F00058206D7574696E672100546F67676C6570
:10020000642074656C656D65747279210050726F3D
:10021000746F636F6C206572726F72207769746897
:100220002052580054696D656F7574207768656E4B
:1002300020636F6E6E656374696E6720746F205201
:100240005800507265737320616E79206B65792058
:10025000746F2063616E63656C00436F6E6E6563DF
:1002600074696E6720746F2052582C20706F776508
:100270007220757020746865205258202877697440
:10028000682062696E6420706C7567206966206EF4
:100290006F74207573696E6720616C776179732064
:1002A00062696E642900546F67676C656420276912
:1002B0006D6D656469617465206F75747075742700
:1002C00000546F67676C65642027736C61766520E6
:1002D0006D6F64652700546F67676C6564202761E4
:1002E0006C776179732062696E642700546F676769
:1002F0006C65642050504D206368616E6E656C20A3
:100300006C696D69740053657420525353492069B8
:100310006E6A656374696F6E206368616E6E656C8A
:100320002028303D3D64697361626C652900536526
:10033000742050504D206D696E696D756D20737914
:100340006E630053657420626561636F6E20696E31
:1003500074657276616C0053657420626561636FC9
:100360006E2064656C617900536574206265616319
:100370006F6E206672657175656E637920696E2097
:10038000487A3A20303D64697361626C652C205074
:10039000783D504D52206368616E6E656C20782CFC
:1003A0002046783D465253206368616E6E656C202E
:1003B00078005365742050574D2073746F7020641B
:1003C000656C61792028302064697361626C6564B2
:1003D0002C20312D323535203D3D20302E317320FB
:1003E0002D2035306D696E29005365742050504DB5
:1003F0002073746F702064656C61792028302064EC
:10040000697361626C65642C20312D323535203D75
:100410003D20302E3173202D2035306D696E29003E
:10042000536574206661696C736166652064656CF0
:1004300061792028302064697361626C65642C20C6
:10044000312D323535203D3D20302E3173202D2089
:1004500035306D696E29002A2A2A2A2A2A2A2A2A50
:100460002A2A2A2A2A2A2A2A2A2A2A2A2A2A2A2AEC
:100470002A2A2A2A0052582041636B6564202D20C5
:1004800072657665727420737563636573736675E0
:100490006C21002A2A2A2A2A2A2A2A2A2A2A2A2AAD
:1004A0002A2A2A2A2A2A2A2A2A2A2A2A2A2A2A2AAC
:1004B000002A2A2A2A2A2A2A2A2A2A2A2A2A2A2AC6
:1004C0002A2A2A2A2A2A2A2A2A2A2A2A2A2A00528E
:1004D000582041636B6564202D20757064617465DC
:1004E000207375636365737366756C21002A2A2A0D
:1004F0002A2A2A2A2A2A2A2A2A2A2A2A2A2A2A2A5C
:100500002A2A2A2A2A2A2A2A2A2A0056616C696457
:100510002063686F69636573206172653A205B319F
:100520005D2D5B31365D20286368616E6E656C20E1
:10053000312D31362900536574206F7574707574D0
:1005400020666F7220706F727420005B585D2061AE
:10055000626F7274206368616E67657320616E6498
:10056000206578697420525820636F6E6669670051
:100570005B535D20736176652073657474696E6783
:100580007320746F205258005B525D20726576654F
:1005900072742052582073657474696E6773207486
:1005A0006F2064656661756C747300557365206EA9
:1005B000756D62657273205B312D445D20746F2010
:1005C0006564697420706F727473205B452D515D92
:1005D00020666F722073657474696E677300202DD6
:1005E00020726563656976657220636F6E66696700
:1005F000757261746F722C20727820737720000AF4
:100600000A6F70656E4C52536E67200053657420FC
:1006100073657269616C2062617564726174653AB8
:10062000200056616C69642063686F696365733A82
:100630002031202D20342B34202F2032202D203823
:10064000202F2033202D20382B34202F2034202D14
:10065000203132202F2035202D2031322B34202FF5
:100660002036202D20313600536574204368616E9A
:100670006E656C20636F6E6669673A20005365741F
:100680002044617461726174652028302D32293AEA
:10069000200053657420486F70206368616E6E653A
:1006A0006C7320286D61782032342C207365706162
:1006B000726174656420627920636F6D6D61732966
:1006C0002076616C69642076616C75657320312DCC
:1006D0003235353A2000536574206368616E6E656B
:1006E0006C2073706163696E6720287831306B48C5
:1006F0007A293A200053657420524620706F77653E
:10070000722028302D37293A200053657420524634
:10071000206D6167696320286865782920652E67E8
:100720002E20307844454144463030443A2000532E
:1007300065742062617365206672657175656E63AC
:10074000792028696E20487A293A20005B5A5D207A
:10075000656E746572207265636569766572206383
:100760006F6E66696775726174696F6E2075746902
:100770006C79005B465D20646973706C61792061FF
:10078000637475616C206672657175656E63696509
:10079000732075736564005B525D2063616C6375E3
:1007A0006C6174652072616E646F6D206B65792079
:1007B000616E6420686F70206C697374005B495DC2
:1007C000207265696E697469616C697A6520736508
:1007D0007474696E677320746F20736B65746368DB
:1007E0002064656661756C7473005B585D2072658A
:1007F00076657274206368616E67657320616E64EC
:100800002065786974206D656E75005B535D20739B
:100810006176652073657474696E677320746F20E8
:10082000454550524F4D20616E64206578697420B3
:100830006D656E7500557365206E756D62657273BA
:10084000205B302D395D20746F20656469742070E1
:100850006172616D657465727300202D2053797328
:1008600074656D20636F6E66696775726174696F18
:100870006E000A0A6F70656E4C52536E672000510D
:1008800029204F7574707574206265666F726520DB
:100890006C696E6B20283D465329203A2000502970
:1008A00020536C617665206D6F64652028657870D3
:1008B0006572696D656E74616C293A20004F29205C
:1008C00054696D65642042494E44206174207374FC
:1008D000617274757020203A20004E292050504DCE
:1008E000206F7574707574206C696D69746564200F
:1008F000202020203A200044495341424C454400E6
:100900004D292050504D205253534920746F20637D
:1009100068616E6E656C202020203A20004C2920F2
:1009200050504D206D696E696D756D2073796E63E1
:10093000202875732920203A200044495341424C15
:100940004544004B29204661696C736166652062ED
:100950006561636F6E20696E74762E2028312D32AA
:10096000353573293A20004A29204661696C736144
:10097000666520626561636F6E2064656C617920D5
:1009800028302D323535203D3E20313073202D204A
:100990003135306D696E293A200049292046616958
:1009A0006C7361666520626561636F6E206672714B
:1009B0002E203A200048292050574D2073746F7024
:1009C0002064656C6179202020202020203A2000BE
:1009D00047292050504D2073746F702064656C61FE
:1009E00079202020202020203A200046292046611E
:1009F000696C736166652064656C617920202020D4
:100A00002020203A200050574D206368616E6E65AB
:100A10006C200066756E6374696F6E3A2000292041
:100A2000706F72742000506F776572546F776572C3
:100A300000445446205548462033322D62697420C4
:100A400031306368004F70656E4C52536E67525878
:100A5000206D696E6920342F36636800466C7974A6
:100A6000726F6E2F4F72616E6765525820554846FF
:100A70002038636800525820747970653A20004429
:100A8000697361626C656400487A00203D3D200016
:100A900043616C63756C61746564207061636B6540
:100AA0007420696E74657276616C3A200042292068
:100AB0004D6963726F202868616C66292050504D23
:100AC000202020203A00412920496E766572746505
:100AD000642050504D20696E20202020203A0030A4
:100AE00029204D7574652062757A7A657220286DAB
:100AF0006F73746C79293A003929205365726961E2
:100B00006C2062617564726174653A00736D617224
:100B100074506F7274004672536B79005472616E38
:100B200073706172656E740044697361626C6564B0
:100B30000038292054656C656D657472793A2020FF
:100B40002020202020003729204368616E6E656CCC
:100B500020636F6E6669673A202000362920446161
:100B60007461726174652028302D32293A2020206A
:100B700000352920486F70206368616E6E656C7364
:100B80003A2020202020003429204368616E6E65C1
:100B90006C2073706163696E673A202000332920EE
:100BA000524620706F7765722028302D37293A2001
:100BB0002020003229205246206D616769633A2067
:100BC0002020202020202020003129204261736530
:100BD000206672657175656E63793A202020000089
:100BE00000000700020100000304060000000000EE
:100BF00000000001020408102040800102040810D7
:100C00002001020408102004040404040404040263
:100C10000202020202030303030303000000002395
:100C2000002600290000000000250028002B0000FD
:100C3000000000240027002A0000352D11241FBECB
:100C4000CFEFD8E0DEBFCDBF13E0A0E0B1E0E8E732
:100C5000F0E602C005900D92A83CB107D9F716E066
:100C6000A8ECB3E001C01D92AC38B107E1F71CE07D
:100C7000CCE3DCE004C02297FE010E943E2ECA3382
:100C8000D107C9F70E94712D0C943A300C940000E2
:100C900080917105813019F482E080937105809113
:100CA0007105833019F484E0809371050895A89547
:100CB0000895DC01ED91FC910190F081E02D099502
:100CC00008952091720530917305382748E0C901D5
:100CD000880F991F37FF06C09C0151E2252750E17C
:100CE000352701C09C01415091F730937305209343
:100CF0007205089588E38093740580E092ECA1E08A
:100D0000B0E08093750590937605A0937705B09336
:100D1000780587E08093810580EC9AECA9E8B6E33A
:100D20008093790590937A05A0937B05B0937C0519
:100D300085E0809382058DEE9EEFADEABEED809357
:100D40007D0590937E05A0937F05B0938005E3E831
:100D5000F5E080E090E0863028F4DC01AE54BC4F32
:100D60002C9101C020E0219301968831910599F7DB
:100D700082E080939B058AE080939C05089580EC37
:100D800097EFAAEBB7E38093B9059093BA05A093C8
:100D9000BB05B093BC0580E090E0A0E0B0E5809397
:100DA000BD059093BE05A093BF05B093C005E1ECCF
:100DB000F5E080E081938F5F8031E1F70895A0E056
:100DC000B0E0E5EEF6E00C94072ED82F0E946C28D8
:100DD0006115710581059105C9F30E94AA2E109233
:100DE0007D0510927E0510927F0510928005C4E06B
:100DF000812C912C54018A94C0907D05D0907E0561
:100E0000E0907F05F0908005FE2CED2CDC2CCC24AE
:100E10000E94A52EA50194010E94E62D6C0D7D1D5A
:100E20008E1D9F1D60937D0570937E0580937F05C9
:100E300090938005C15001F7DD2309F450C003E809
:100E400015E0E801A12CB12C62E3C62ED12CE12CD7
:100E5000F12C8881882309F442C0B39419F40E94CC
:100E60007A063DC00E94A52EA70196010E94E62D9C
:100E7000E1E0E60FA3E8B5E08A2F801B8A1520F495
:100E80008D918E13F9CFE9CF2091820530E0A0E15A
:100E9000B7E20E947E2D9B01AC01AE2FB0E00E9414
:100EA0008D2D4090790550907A0560907B0570906B
:100EB0007C05640D751D861D971D4090B9055090E9
:100EC000BA056090BB057090BC05461657066806CB
:100ED000790618F2E993A39488E1A812BACFCDB7A6
:100EE000DEB7E0E10C94232E8436910520F4BC019A
:100EF00080E090E017C09C018E3B910528F42A55B4
:100F00003109AAE0B0E00CC0823D910528F4245BD1
:100F10003109A4E6B0E004C02D5C3109A8E5B2E0D7
:100F20000E947E2DA4E6B0E09B01AC010E948D2DB5
:100F3000089590E08C599F4F0E947407089561E0D6
:100F40008AE00E94192960E08AE00E9452290895EF
:100F5000892B11F061E001C060E08AE00E94522913
:100F6000089560E089E00E94192961E088E00E940C
:100F7000192961E087E00E94192960E082E00E945F
:100F8000192961E084E00E941929089542E050E0A7
:100F900068E476E080E00E949C270895E3E0F0E0BA
:100FA00089E080935700E491E67081E0E63009F033
:100FB00080E00895CF93DF93C82F0E94CE07882347
:100FC00081F0DFB781E080937005F8940E945706A6
:100FD00088E180936000C0936000C1110E945706B1
:100FE000DFBFDF91CF9108958F929F92AF92BF9212
:100FF000CF92DF92EF92FF92CF93FC01C0A5EC2F2E
:10100000E770F0E0E658FC4FA081B0E0C7FF03C0F6
:1010100024E130E002C02FE030E0FC0197A183E141
:10102000989FF0011124E25CFE4F80809180A280A5
:10103000B380A20FB31F20E43FE14DE750E00E94D0
:10104000982DA50194010E94C42D8C2F887149F41C
:1010500069017A01E0EDCE0EE7E0DE1EE11CF11C35
:101060001BC0C7FF05C060E47AE88CE29EE004C0C4
:1010700060E07EEE8AEB9BE069017A01F8EBCF0E2F
:10108000FBE0DF1EE11CF11CA50194010E94C42DB0
:10109000C20ED31EE41EF51EC701B60169517C4F76
:1010A0008F4F9F4F28EE33E040E050E00E94C42D68
:1010B000A8EEB3E00E948D2DCF91FF90EF90DF90CE
:1010C000CF90BF90AF909F908F9008958F3F9105E4
:1010D00051F048F0811522E0920738F081159340D5
:1010E00030F482E0089580E0089581E0089583E07F
:1010F0000895A0E0B0E0EFE7F8E00C94102EEB01CB
:101100008A01B82FB695A0E028813981F8012083A3
:101110002A813B8121832C813D8122832E813F8145
:101120002383688179814A815B812C813D81EE81B5
:10113000FF819F2F9295990F990F907C272F2370F5
:10114000922B252F2370220F220F922B232F2370F7
:101150002295207F922BF80194830B5F1F4F2896D6
:10116000AF5FBA1788F680FF24C0888199810E94FA
:101170006608D82E8A819B810E946608E82E8C81A1
:101180009D810E946608F82E8E819F810E946608CC
:10119000F0E4DF9EA001112490E1E99E900111246A
:1011A000242B282BE4E0FE9EB0011124262BF8010D
:1011B0002083CDB7DEB7E7E00C942C2E803223E0FD
:1011C000920708F1883E23E0920740F48F51934044
:1011D000E4E096958795EA95E1F70895803D27E04C
:1011E000920718F48C5D93400895883928E092079F
:1011F00068F4885C974074E0969587957A95E1F756
:101200008D509C4F089580E090E008958FEF93E01B
:1012100008958C30910540F4A4E0880F991FAA9599
:10122000E1F7885D9C4F0895843F23E0920718F40E
:1012300084529C4F0895811524E0920740F486570C
:10124000934FF4E0880F991FFA95E1F7089580E92C
:1012500098E008959C013695279525753575821B74
:10126000930B9C0123733373969587959695879579
:1012700083739373820F931F9C0154E036952795D7
:101280005A95E1F7280F391F2F703F7041E051E068
:10129000249FC001259F900D349F900D1124892F0C
:1012A00008955F98882319F00000289A02C0000072
:1012B000289800005F9A000008955F9A000083B1AB
:1012C0005F980000869581700895CF93DF93D82FA3
:1012D0005C9A5F985C98C8E08D2F80780E945109D5
:1012E000DD0FC150C9F75F98DF91CF9108958F77D7
:1012F0000E9465090895CF93DF93D82FC8E08D2F02
:1013000080780E945109DD0FC150C9F75F98DF91C5
:10131000CF910895CF93DF935F98C8E080E0D82FF6
:10132000DD0F0E945D098D0FC150C9F7DF91CF918C
:1013300008950E9477090E948A095C9A0895A1E0A5
:10134000B0E0E5EAF9E00C94152E806869830E940C
:1013500065096981862F0E947B095C9A2196E2E0EB
:101360000C94312ECF93C0917D05C827E82FF0E073
:10137000EC58FA4F678589E70E949F096C2F8DE32F
:101380000E949F096C2F82E40E949F09CF910895CB
:1013900086E20E9499090895CF93DF93EC016C8156
:1013A0008CE10E949F096D818DE10E949F096E81F1
:1013B0008EE10E949F096F8180E20E949F096885EB
:1013C00081E20E949F09698582E20E949F096A85E5
:1013D00083E20E949F096B8584E20E949F096C85CD
:1013E00085E20E949F096D858AE20E949F096E85B1
:1013F0008EE60E949F096F858FE60E949F0968898B
:1014000080E70E949F09698981E70E949F096A8994
:1014100082E70E949F09DF91CF910895CF92DF92DA
:10142000EF92FF92CF93DF936B017C01C11488E3AD
:10143000D8068CE9E8068CE1F80628F5C701B60164
:1014400020E836E948E950E00E94C42DE901689798
:1014500060E879E687E69FEF0E94A02D6C0D7D1D68
:101460008E1D9F1DF2E0660F771F881F991FFA954A
:10147000D1F721E732E040E050E00E94C42DF22E87
:10148000E32E80E421C0C701B60120E03DE241E344
:1014900051E00E94C42DE901689760E073ED8EEC85
:1014A0009EEF0E94A02D6C0D7D1D8E1D9F1D660F51
:1014B000771F881F991F21E732E040E050E00E942B
:1014C000C42DF22EE32E80E66C2F6F71680F85E736
:1014D0000E949F096E2D86E70E949F096F2D87E766
:1014E0000E949F09DF91CF91FF90EF90DF90CF9006
:1014F0000895682F8DE60E949F0908958F929F920C
:10150000AF92BF92CF92DF92EF92FF92CF93DF9391
:10151000D82F83E00E94990980936F0584E00E9490
:10152000990980936E0560E086E00E949F0961E062
:1015300087E00E949F096FE789E00E949F0965E0AC
:101540008AE00E949F0962E18BE00E949F0965E1A9
:101550008CE00E949F096DEF8DE00E949F0960E082
:101560008EE00E949F09DD2319F08BE291E008C014
:1015700020919B0533E1239FC0011124825C9E4F83
:101580000E94CC096CE880E30E949F096FE082E32F
:101590000E949F0962E483E30E949F0980919C0559
:1015A00087FF02C064E101C06AE084E30E949F09F2
:1015B0006AE285E30E949F096DE286E30E949F092B
:1015C00064ED87E30E949F0960E088E30E949F0921
:1015D00060E089E30E949F09D11109C0C0907D0598
:1015E000D0907E05E0907F05F090800507C0C5E9AA
:1015F000CC2EC1ECDC2EED2CCEEDFC2ECAE38F2CD4
:101600009924AA24BB24682D8C2F0E949F09682D41
:1016100085E08C0F0E949F09FE2CED2CDC2CCC2445
:10162000CF5FCE3361F76FEF83E40E949F096FEFC6
:1016300084E40E949F096FEF85E40E949F096FEF89
:1016400086E40E949F09DD2311F066E002C06091EC
:1016500081058DE60E949F0960E089E70E949F094D
:10166000609182058AE70E949F0960E083E70E94FB
:101670009F0960E084E70E949F09D11109C0609131
:10168000790570917A0580917B0590917C0504C065
:1016900060EC7AEC89E896E30E940E0ADF91CF9124
:1016A000FF90EF90DF90CF90BF90AF909F908F9082
:1016B000089561E087E00E949F0964E28EE70E943E
:1016C0009F0963E088E00E949F0960E088E00E9433
:1016D0009F0965E087E00E949F0962E085E00E9423
:1016E0009F0983E00E94990980936F0584E00E941E
:1016F000990980936E05089583E00E94990980936B
:101700006F0584E00E94990980936E0561E087E08F
:101710000E949F096AE070E080E090E00E948F28BC
:101720000E94590B00000895CF92DF92FF920F9311
:101730001F93CF93DF931F92CDB7DEB7082F162FDD
:101740008EE399830E949F09F02EC02E9981D92E95
:101750008C2D8F19811738F4F60161916F018FE795
:101760000E949F09F5CF64E085E00E949F0983E015
:101770000E94990980936F0584E00E9499098093E3
:101780006E050E946C2860936A0570936B058093C8
:101790006C0590936D0569E087E00E949F0981E0E8
:1017A000809371050F90DF91CF911F910F91FF9062
:1017B000DF90CF9008950F931F930E94940B809118
:1017C0007105813099F40E946C2800916A0510918E
:1017D0006B0520916C0530916D05601B710B820BC0
:1017E000930B603A76488140910548F380917105EA
:1017F000813031F46EE971E080EE95E00E94582A64
:101800001F910F9108950F931F938091710582305E
:1018100021F41092710581E020C080917105813022
:10182000D9F40E946C2800916A0510916B052091F3
:101830006C0530916D05601B710B820B930B613A47
:1018400076488140910540F061E087E00E949F0961
:101850001092710582E001C080E01F910F91089500
:10186000CF93DF93EC014AE050E06D2F70E080EE03
:1018700095E00E94262B6EE280EE95E00E942A2AD7
:10188000BE0184E0769567958A95E1F76F707727BA
:101890004AE050E080EE95E00E94262BDF91CF9148
:1018A0000895D82FC0E0CD1780F42D9A64E670E03B
:1018B00080E090E00E948F282D9864E670E080E040
:1018C00090E00E948F28CF5FEECF6CE271E080E065
:1018D00090E00E948F28E6CF0F931F93CF93DF9362
:1018E000EC01062F15E0115051F0CE010E9421307D
:1018F000081741F0602FCE010E942930F4CF82E01A
:101900000E94510CDF91CF911F910F910895A0E09B
:10191000B0E0EDE8FCE00C94072E482E562EC0E017
:10192000D0E0612C712CE12CF12C00E010E0411092
:101930000CC06090D20586E4689E3001112459E104
:10194000E52EF12C08EB15E01EC091E049120FC006
:101950006090D205E6E46E9E30011124FBE16F0E2B
:10196000711C49E2E42EF12C04E715E00CC082E082
:10197000481209C028E1622E77247394EE24E39480
:10198000F12C01ED15E043018C0E9D1E10927305A4
:10199000109272053401A62CA818B12CC30101962F
:1019A0006C01AE14BF04A8F4A00EB11E511006C005
:1019B000C3010E942130F501808305C0F5016081DB
:1019C000C3010E946C0CF50180810E946106360102
:1019D000E2CFC301511018C0C3010E942130B82EBC
:1019E000C6010E9421302B2D30E0322F2227282BD8
:1019F00080917205909173058217930779F4C0E086
:101A0000D0E05524539493CF3601609173050E9422
:101A10006C0C60917205C6010E946C0CC05EDE4FBA
:101A2000C13E92E0D90708F482CF852DCDB7DEB74D
:101A3000E0E10C94232E61E082E00E94870C08957F
:101A400060E082E00E94870C8091D105853028F00B
:101A500084E08093D1050E941B0D8091D105809375
:101A6000D205089561E080E00E94870C61E081E08A
:101A70000E94870C089560E080E00E94870C882314
:101A800051F060E081E00E94870C882321F0809172
:101A90007405883349F00E94BF060E947A0681E0EF
:101AA0000E94DF060E94320D0895882319F06AEA29
:101AB00071E002C06EEA71E080EE95E00E94582A63
:101AC0000895FF920F931F93CF93DF9369EC7BE010
:101AD00080EE95E00E94042A4091790550917A05A4
:101AE00060917B0570917C052AE030E080EE95E006
:101AF0000E942D2B63EB7BE080EE95E00E94042A90
:101B000040917D0550917E0560917F057091800523
:101B100020E130E080EE95E00E942D2B6DE97BE026
:101B200080EE95E00E94042A4AE050E06091810531
:101B300080EE95E00E94552B67E87BE080EE95E013
:101B40000E94042A4AE050E06091820580EE95E010
:101B50000E94552B61E77BE080EE95E00E94042A0D
:101B6000C3E8D5E0F12C8E0188818823A9F0FF20FD
:101B700031F061EB71E080EE95E00E94272A21961A
:101B80004AE050E0F801608180EE95E00E941E2B53
:101B9000F394F8E1FF12E7CF80EE95E00E94322A3D
:101BA0006BE57BE080EE95E00E94042A4AE050E07D
:101BB00060919B0580EE95E00E94552B66E47BE0EA
:101BC00080EE95E00E94042AE0919C05E770F0E029
:101BD000EE0FFF1FEE57FC4F6081718180EE95E0A4
:101BE0000E94582A61E37BE080EE95E00E94042A7F
:101BF00080919C058871883069F028F4811113C0A8
:101C000068E27BE00CC0803141F0883161F46CE027
:101C10007BE005C06CE17BE002C066E17BE080EE2A
:101C200095E00E94462A68EF7AE080EE95E00E94F7
:101C3000042A409175055091760560917705709161
:101C400078052AE030E080EE95E00E942D2B6FEDC4
:101C50007AE080EE95E00E94042A8091BD058071B3
:101C60000E94550D66EC7AE080EE95E00E94042A11
:101C70008091BD0580740E94550D6DEA7AE080EE7A
:101C800095E00E94042A8091BD0580720E94550D46
:101C900060E97AE080EE95E00E94042A84E795E00E
:101CA0000E94F407AB01BC012AE030E080EE95E031
:101CB0000E940F2B6BE87AE080EE95E00E94042AE8
:101CC00084E795E00E94F4079B01AC0160E472E4B4
:101CD0008FE090E00E94C42DBA01A9012AE030E013
:101CE00080EE95E00E940F2B68E87AE080EE95E0A8
:101CF0000E94462ACDB7DEB7E5E00C942E2E8F92D7
:101D00009F92AF92BF92CF92DF92EF92FF9281119A
:101D100007C06FE77AE080EE95E00E94462A2FC068
:101D200090E00E94740724E630E040E050E00E941A
:101D3000C42DCA01B9012AE030E040E050E00E9421
:101D4000C42D49015A016B017C012AE030E0B50144
:101D5000A40180EE95E00E940F2B6EE280EE95E0EC
:101D60000E942A2A2AE030E0B701A60180EE95E021
:101D70000E940F2B63E780EE95E00E946A2AFF9095
:101D8000EF90DF90CF90BF90AF909F908F9008958D
:101D90001F93CF93DF9365E77AE080EE95E00E9492
:101DA000042A80919D05813041F46CE57AE080EE53
:101DB00095E00E94462A10E050C0823019F465E494
:101DC0007AE0F5CF843019F461E37AE0F0CF853022
:101DD00091F766E27AE0EBCFC12FD0E0C930D105B0
:101DE0000CF441C068E3610F80EE95E00E942A2A5E
:101DF0006EE17AE080EE95E00E94042ABE016F5FFA
:101E00007F4F4AE050E080EE95E00E94EE2A63E1C9
:101E10007AE080EE95E00E94042AC356DA4FE98109
:101E2000E03218F566E07AE080EE95E00E94042A40
:101E30008981803130F06DE673E080EE95E00E949C
:101E4000272A69816F7070E06F5F7F4F4AE050E032
:101E500080EE95E00E94F72A1F5F809146051817D3
:101E600008F4BACF0FC061E3BECFEF70F0E0EE0F21
:101E7000FF1FEE56FC4F6081718180EE95E00E945D
:101E8000582AEACF6BEE79E080EE95E00E94042AB2
:101E90008091B5050E947F0E60ED79E080EE95E0BF
:101EA0000E94042A8091B6050E947F0E65EB79E0BE
:101EB00080EE95E00E94042A8091B7050E947F0E73
:101EC0006AE979E080EE95E00E94042A4091AD0530
:101ED0005091AE056091AF057091B0054115510567
:101EE0006105710539F12AE030E080EE95E00E944D
:101EF0002D2B67E679E080EE95E00E94042A809120
:101F0000B1050E949907AB01BC012AE030E080EEE8
:101F100095E00E942D2B63E479E080EE95E00E942D
:101F2000042A4AE050E06091B20580EE95E00E94FC
:101F3000552B06C06AE379E080EE95E00E94462AC0
:101F40006DE179E080EE95E00E94042A6091B3058E
:101F50007091B4054AE050E080EE95E00E943F2B7E
:101F600060E079E080EE95E00E94042A6091AC0583
:101F7000603450F470E06F5F7F4F4AE050E080EED5
:101F800095E00E94F72A06C067EF78E080EE95E0C2
:101F90000E94462A6AED78E080EE95E00E94042ACD
:101FA0008091AB0580FF03C063EB71E002C067EB7B
:101FB00071E080EE95E00E94582A6DEB78E080EEAB
:101FC00095E00E94042A8091AB0582700E94550D15
:101FD0006EE978E080EE95E00E94042A8091AB05DE
:101FE00084700E94550D6FE778E080EE95E00E94C6
:101FF000042A8091AB0588700E94550DDF91CF9126
:102000001F9108950F931F93CF93DF932091430562
:102010002F3FA9F56FEF75E080EE95E00E94042A4E
:1020200080E893E00E94300C6EED75E080EE95E064
:102030000E94042A80914405909145050E94300C2D
:102040006BEA75E080EE95E00E94462A68E875E04C
:1020500080EE95E00E94462A60E775E080EE95E00C
:102060000E94462A6BE475E080EE95E00E94462AC5
:1020700080EE95E00E94322A0E94C80E68C01216B7
:102080000CF065C0332727FD30958091460590E020
:10209000821793070CF45BC066E375E080EE95E071
:1020A0000E94042A60914305772767FD70954AE0F6
:1020B00050E080EE95E00E94F72A6BE075E080EE3C
:1020C00095E00E94042A10E008E280914705181765
:1020D000D0F5C12FD0E0CC0FDD1FC85BDA4F2881CF
:1020E00030E080914305992787FD90950197281747
:1020F000390739F56BEB71E080EE95E00E94272AF5
:102100004AE050E0602F80EE95E00E941E2B6FEBBE
:1021100071E080EE95E00E94272AE981EF70F0E0FF
:10212000EE0FFF1FEE56FC4F6081718180EE95E04F
:102130000E94272A63EC71E080EE95E00E94272A36
:102140000F5F1F5FC2CF80EE95E00E94322ADF91C1
:10215000CF911F910F910895FF920F931F93CF93EB
:10216000DF93C3E8D5E0F12C8E0188818823D1F17B
:1021700065EC71E080EE95E00E94272A4AE050E08D
:102180006F2D80EE95E00E941E2B62ED71E080EED7
:1021900095E00E94272A2196F801208130E0A0E1F5
:1021A000B7E20E947E2D9B01AC01A0918205B0E0B8
:1021B0000E948D2DAB01BC018091790590917A052B
:1021C000A0917B05B0917C05480F591F6A1F7B1FAA
:1021D0002AE030E080EE95E00E942D2BF394F8E1A8
:1021E000FF12C2CFCDB7DEB7E5E00C942E2E1092D1
:1021F000DD0485E6EEEDF4E0DF011D928A95E9F756
:102200000895CF93C82F8F3719F0883009F045C053
:10221000E091DD04EE23D9F1E150E093DD04F0E03C
:10222000E252FB4F10826DE070E080EE95E00E947C
:102230005906C0E08091DD04C81760F4EC2FF0E08F
:10224000E252FB4F608170E080EE95E00E945906FB
:10225000CF5FF0CF60E270E080EE95E00E9459061B
:102260006DE070E080EE95E00E945906C0E080913C
:10227000DD04C81778F5EC2FF0E0E252FB4F6081E7
:1022800070E080EE95E00E945906CF5FF0CF67E0E6
:1022900080EE95E00E942A2A1DC08B3119F40E941D
:1022A000F7101AC08D30C1F08A30B1F08091DD0492
:1022B000843668F76C2F70E080EE95E00E94590636
:1022C000E091DD0481E08E0F8093DD04F0E0E252C6
:1022D000FB4FC08380E001C081E0CF910895CF9390
:1022E000C82F0E946C286093C6047093C704809323
:1022F000C8049093C904C093DB04CC2329F040E0C8
:1023000051EE60E070E004C040E855E260E070E04B
:1023100080EE95E00E94B42CCF9108959091CA046C
:10232000492F4F7050E0BA016F5F7F4F292F30E087
:10233000E4E035952795EA95E1F76217730759F0C0
:10234000FA01E553FB4F808381E0890F8F70907F06
:10235000892B8093CA0408956EE770E080EE95E0C3
:102360000E9459060895A3E1B1E0E9EBF1E10C9474
:10237000082EE3E8F5E0712C8191882321F0739415
:1023800028E17212F9CF66ED71E080EE95E00E94CF
:10239000582A4AE050E0672D80EE95E00E94552BC8
:1023A00080E00E947E0A0E94590B8E010E5F1F4F33
:1023B000C12CD12C7601C39466246A945C2C0E94B3
:1023C00060284B015C012091820530E0A0E1B7E27A
:1023D0000E947E2D9B01AC01C701B6010E94A02D79
:1023E0002091790530917A0540917B0550917C05CB
:1023F000620F731F841F951F2091B9053091BA0594
:102400004091BB055091BC0526173707480759076F
:1024100018F4F801608225C08C2D0E94B20961E099
:1024200070E080E090E00E948F28F80110820E9406
:102430006028681979098A099B09643F7140810500
:10244000910540F40E94C809F8019081981778F727
:102450008083EDCF50FE03C02C982D9A02C02C9A99
:102460002D982FEFC21AD20AE20AF20A0F5F1F4F0D
:102470008FEFC816D104E104F10409F09FCFCE011B
:102480009395FC01D82E7FEF68EC2E2F281B271583
:1024900010F051E056C0DE01129651E02FEF41E0FE
:1024A0003D91321710F0322F01C0452F5F5F5F3F23
:1024B00011F0232FF5CF4193242F30E0A1E0B0E0BD
:1024C000AC0FBD1FA20FB31F5C93413079F0DE014A
:1024D000A20FB31F5C93423049F0AFEFBFEFAC0FD8
:1024E000BD1FA20FB31F6C934E3F78F6A2E0B0E081
:1024F000AC0FBD1FA20FB31F7C934D3F30F6A3E07E
:10250000B0E0AC0FBD1FA20FB31F6C93BECF452F21
:10251000242F30E0FC01E20FF31F6081AFEFB0E049
:10252000AC0FBD1FA20FB31F2C91621748F441508E
:10253000DC01A40FB11D2C9120836C934111E8CFD5
:102540005F5F571520F3372D369520E0231770F481
:10255000DC01A20FB11D4C91522F530FFC01E50F6E
:10256000F11D50815C9340832E5FF0CFF3E8EF2E96
:10257000F5E0FF2E8C01802F8D19871598F4F80156
:10258000C1908F014AE050E06C2D80EE95E00E94F2
:102590001E2B6CE280EE95E00E942A2AF701C19280
:1025A0007F01E9CF80EE95E00E94322A81E0CD5E86
:1025B000DE4FEFE00C94242E1F920F920FB60F9275
:1025C00011240F931F932F933F934F935F936F9318
:1025D0007F938F939F93AF93BF93EF93FF9340911C
:1025E000BD055091BE056091BF057091C00589B1D0
:1025F0008A019B01007411272227332783FB882738
:1026000080F990E0A0E0B0E0081719072A073B071F
:1026100009F468C080918400909185001092850033
:10262000109284002091A70421115CC045FD02C0D6
:1026300096958795853C29E09207C0F180910A0123
:1026400090E0A0E0B0E00CE176956795579547954E
:102650000A95D1F7411551056105710521F441E055
:1026600050E060E070E0481759076A077B07D8F42C
:1026700080910A018F3FB9F040E080910A0148172C
:1026800080F4842F90E0880F991FFC01E957FB4FDD
:1026900020813181FC01E55FFE4F318320834F5F54
:1026A000ECCF1092A80410920A011CC08D3B22E0CE
:1026B0009207A8F020910A01203188F410910A01B4
:1026C00021E0210F20930A010E94DE08E12FF0E0B3
:1026D000EE0FFF1FE957FB4F9183808303C08FEFFD
:1026E00080930A01FF91EF91BF91AF919F918F91DC
:1026F0007F916F915F914F913F912F911F910F911A
:102700000F900FBE0F901F90189583E0809380006C
:102710008AE1809381008FEF9FEF909389008093EF
:10272000880010926F0088E080936D00E8E6F0E08A
:1027300080818460808308950E94200D8091D2055D
:10274000843011F41092D20508956F3018F08695F8
:102750008058089589E0689F802D11240895A0E095
:10276000B0E0E5EBF3E10C940F2EC82F0E946C282B
:10277000009138041091390420913A0430913B04BF
:102780006B017C01C01AD10AE20AF30A97018601A3
:1027900049E8C41643E1D406E104F10410F01092B4
:1027A0003C04609338047093390480933A04909306
:1027B0003B042091A7048FEF820F8230D8F5E0917F
:1027C0003C04EE2309F44EC1E13011F482E0B8C1BB
:1027D000E03108F034C181E08E0F80933C04F0E0DA
:1027E000E957FB4FC083803109F0ACC1E9E8F4E060
:1027F000213029F4A181A695A695808108C0808109
:102800009181A92FA695A695A69596958795A03115
:1028100048F4B0E090E0AA0FBB1FA55FBE4F119631
:102820009C938E931092A804329684E0E739F807BF
:10283000F9F688C1233009F005C1E0913C04E111AB
:1028400004C0CF3009F07EC10DC1E83148F481E009
:102850008E0F80933C04F0E0EA57FB4FC08372C1B7
:10286000E83109F0ECC0C111EAC040E050E0ABE053
:10287000CA01B3E0880F991FBA95E1F7A49F9001B0
:10288000A59F300D1124F901E957FB4F6081E181CB
:102890007E2F777075956795FC01EE0FFF1FE55F42
:1028A000FE4F71836083F901E857FB4FB081B69505
:1028B000B695B695E181FE2FF295FF0FF07E6F2F52
:1028C0006B2BE695E695E6957E2F77707595679567
:1028D000FC01EE0FFF1FE35FFE4F71836083F90180
:1028E000E757FB4FB081B295B695B695B370C181ED
:1028F000DC2FDD0FDD0F6D2F6B2BC295C695C695B6
:10290000C370E281E170EE0FEE0F7E2F7C2B759588
:102910006795FC01EE0FFF1FE15FFE4F718360833F
:10292000F901E557FB4FB081B695E181FE2FF79590
:10293000FF27F7956F2F6B2BE6957E2F7770759598
:102940006795FC01EE0FFF1FEF5EFE4F7183608302
:10295000F901E457FB4FB081B295BF70E181FE2FC2
:10296000F295F07F6F2F6B2BE295EF707E2F7770D3
:1029700075956795FC01EE0FFF1FED5EFE4F7183AD
:102980006083F901E357FB4FB081BB1FBB27BB1F1F
:10299000C181DC2FDD0F6D2F6B2BCC1FCC27CC1F03
:1029A000E281E370EE0F7E2F7C2B75956795FC011D
:1029B000EE0FFF1FEB5EFE4F71836083F901E1575D
:1029C000FB4FB081B695B695E181FE2FF295FF0FD2
:1029D000FF0FF07C6F2F6B2BE695E6957E2F7770BF
:1029E00075956795FC01EE0FFF1FE95EFE4F718341
:1029F0006083F901E057FB4F2081229526952770CF
:102A00003181E32FEE0FEE0FEE0F6E2F622B732F3F
:102A100072957695777075956795FC01EE0FFF1F9F
:102A2000E75EFE4F718360834F5F5F4F4230510519
:102A300009F01ECF80919D0483FF1092A80410928C
:102A40003C0480C0243009F07DC060913C046111D9
:102A50000BC0C83AB1F4109273051092720588EA5F
:102A60000E94610681E06CC0613019F4C0933704A4
:102A700004C0623031F4C09336048C2F0E9461068A
:102A80005AC0E09136042E2F30E0220F331F462F1C
:102A900050E0C9010296841795073CF0633268F74D
:102AA000FA01EC57FB4FC083E8CF2D5F3F4F8C2FCF
:102AB00090E060917205709173054217530749F4D5
:102AC000982F882786279727909373058093720500
:102AD00032C06817790769F580913704813049F56C
:102AE000E13118F080E180933604F0903604C8E8B4
:102AF000D4E000E010E00F15D0F4FE0131978081A2
:102B000090E0982F88272881822B43E0969587951F
:102B10004A95E1F70E94DE08F801EE0FFF1FE55F1E
:102B2000FE4F918380830F5F1F4F2296E4CF109258
:102B3000A80410923C0480913C04882319F08F5F14
:102B400080933C04CDB7DEB7E8E00C942B2EE82F41
:102B5000F0E0E854FA4FE185E03150F4F894F0E009
:102B6000EE0FFF1FE55FFE4F8081918178940895FD
:102B7000E03121F0E13131F483E101C082E10E94D2
:102B8000AE29089580E092E00895A2E2B0E0EBEC77
:102B9000F5E10C94052E9E012F5F3F4F80E1D90196
:102BA0001D928A95E9F764E072E080EE95E029A332
:102BB0003AA30E94582A0E947C0B1D8A1E8A1F8AF3
:102BC000188E312C212C00E0812C912C540170ECBA
:102BD000472E7DE9572E78E5672E75E3772EE0E5E1
:102BE000CE2EE3ECDE2EE12CF12C84EF91E0A0E080
:102BF000B0E08D8F9E8FAF8FB8A380EC97EFAAEBDC
:102C0000B7E3898F9A8FAB8FBC8F80EC9DE9A8E5E5
:102C1000B5E3898B9A8BAB8BBC8B80EE95E00E94E1
:102C20006C2B892B09F4E1C080EE95E00E94992B72
:102C30009C0133272C32310509F442C0ACF4233215
:102C4000310509F0ABC019821A821B821C821D82D9
:102C50001E821F82188619861A861B861C861D8670
:102C60001E861F86188A60C02434310529F023355A
:102C7000310509F4B2C092C064E480EE95E00E9490
:102C80002A2A2AE030E040EC5DE968E575E380EE51
:102C900095E00E94B82A6CE280EE95E00E942A2A14
:102CA0002AE030E040EC57EF6AEB77E380EE95E006
:102CB0000E94B82A6CE280EE95E00E946A2AADCFAD
:102CC0000F5F043009F0A9CF29813A814B815C81E3
:102CD000A8EEB3E00E948D2D698B7A8B8B8B9C8B39
:102CE0002D813E814F8158850E948D2D698F7A8F6D
:102CF0008B8F9C8F29853A854B855C852D8F3E8FE8
:102D00004F8F58A32D853E854F8558890E948D2D64
:102D10006B017C0160323EE473078105910530F45C
:102D200062E38CE10E949F0900E077CF603345E7C2
:102D300074078105910510F462E2F3CF60345CE919
:102D400075078105910510F466E2EBCF80E5C816A2
:102D500083ECD806E104F10410F462E1E2CF90E6DE
:102D6000C9169AEED906E104F10410F465E1D9CF51
:102D7000A0E7CA16A1E1DA06A1E0EA06F10410F420
:102D800061E0CFCFB0EACB16B6E8DB06B1E0EB06E8
:102D9000F10410F463E0C5CF65E0C3CF10ED180F68
:102DA0001A3008F03ACFE1E0F0E0EC0FFD1F24E02C
:102DB000029FE00DF11D1124208131814281538158
:102DC000AAE0B0E00E948D2D610F711D811D911D43
:102DD000608371838283938320CF49885A886B886C
:102DE0007C88812C912C540118CF81149104A1046A
:102DF000B10489F4C301B2010E940E0A61E070E0DF
:102E000080E090E00E948F281D8A1E8A1F8A188EFB
:102E1000312C22242A948D8D9E8DAF8DB8A18816D9
:102E20009906AA06BB06D0F40E94C8092D893E89DE
:102E30004F89588D280F311D411D511D2D8B3E8B03
:102E40004F8B588F381608F4382E821508F4282E28
:102E50003FEF831A930AA30AB30A56C0C301B20113
:102E600028EE33E040E050E00E94C42DBA01A901F1
:102E70002AE030E080EE95E00E940F2B6CE280EEBD
:102E800095E00E942A2A4AE050E0632D80EE95E00A
:102E90000E941E2B6CE280EE95E00E942A2A6D892A
:102EA0007E898F89988DA50194010E94C42DBA0155
:102EB000A9012AE030E080EE95E00E940F2B6CE241
:102EC00080EE95E00E942A2A4AE050E0622D80EED2
:102ED00095E00E941E2B6CE280EE95E00E946A2A2B
:102EE0004C0C5D1C6E1C7F1C898D9A8DAB8DBC8D2E
:102EF00084159505A605B70520F449885A886B887E
:102F00007C88812C912C540129893A894B895C89D0
:102F1000283E33404105510509F07FCEA296E2E1FB
:102F20000C94212EACE1B0E0E8E9F7E10C940F2E0F
:102F30000E946C286B017C0181E00E947E0A14E7EC
:102F400003E0198361E0CE0101960E94DB0B009340
:102F500071050E94590B6AEF70E080E090E00E94DA
:102F60008F2880917105833089F480EE95E00E946E
:102F70006C2B892B59F40E946C286C197D098E09E1
:102F80009F096038734C894C9140D8F2809171054B
:102F9000833009F44FC08FE70E9477090E948A09A5
:102FA0008983843511F083E05CC00E948A09109205
:102FB0004405809345050E948A092091440530917B
:102FC0004505280F311D30934505209344050E9487
:102FD0008A09809346050E948A09809347058131BA
:102FE00010F7F12C0F2D10E08091470590E0880F2D
:102FF000991F0817190740F40E948A09F801E85B35
:10300000FA4F8083F394EECF80E7898361E0CE01AD
:1030100001960E94DB0B83E0809371050E94590B9F
:1030200062E370E080E090E00E948F28809171055B
:10303000833011F482E015C08FE70E9477090E9467
:103040008A098983803509F0AECF0DE915E00E9429
:103050008A09F80181938F01F5E0083B1F07B9F752
:1030600081E06C96E8E00C942B2E80914305992723
:1030700087FD9095A92FB92FFC013196EB30F10512
:1030800008F066C0EC5CFF4F0C943C2E62E778E0E1
:1030900080EE95E00E94462A80E893E00E94300C82
:1030A0006AE578E080EE95E00E94462A65E378E0E4
:1030B00080EE95E00E94462A6BE078E080EE95E095
:1030C0000E94462A6AEE77E080EE95E00E94462A4A
:1030D0006DEB77E080EE95E00E94462A67E977E0A5
:1030E00080EE95E00E94462A63E777E080EE95E067
:1030F0000E94462A6CE477E080EE95E00E94462A22
:1031000080EE95E00E94322A0E94610D21C06FE29C
:1031100077E01AC06AE077E017C065EF76E014C088
:1031200066ED76E011C062E976E00EC06DE776E00C
:103130000BC068E676E080EE95E00E94462A62E2E7
:1031400076E002C06CE076E080EE95E00E94462AD0
:103150006AE070E080E090E00E948F2880EE95E0C9
:103160000E946C2B892B29F080EE95E00E94992B10
:10317000F5CF0895ACE1B0E0E0ECF8E10C940F2E4F
:10318000909143059F3F09F023C1482F50E0FA0179
:103190003A97EF36F10508F00FC1E15CFF4F0C9450
:1031A0003C2E61E172E0A0C06DE172E080EE95E03E
:1031B0000E94582A85E789838BE1EDE9F5E0DE017D
:1031C000129601900D928A95E1F76CE1CE0101967D
:1031D0000E94DB0B0E94590B83E08093710568EC21
:1031E00070E080E090E00E948F288091710584302B
:1031F00009F0E2C08FE70E9477090E948A0989835B
:10320000853509F0D9C06DEE74E080EE95E00E943E
:10321000462A6FEC74E080EE95E00E94462A61EB4E
:1032200074E096C065E372E080EE95E00E94582A53
:1032300089E6898361E0CE0101960E94DB0B0E9442
:10324000590B83E08093710568EC70E080E090E0BA
:103250000E948F2880917105843009F0ADC08FE7FE
:103260000E9477090E948A0989838E010E5F1F4F91
:103270007E014DE1E40EF11C0E948A09F801819360
:103280008F01EE15FF05C1F78BE1FE013296ADE926
:10329000B5E001900D928A95E1F78981893409F0B2
:1032A0008BC063E974E080EE95E00E94462A65E7F2
:1032B00074E080EE95E00E94462A67E574E048C01D
:1032C0006FE472E080EE95E00E94582A8EEF8093C2
:1032D000430572C0805287508053909146059817DD
:1032E00008F066C06EE572E080EE95E00E94582A14
:1032F00063C084E18093430560E274E029C085E106
:103300008093430569EE73E023C086E18093430513
:1033100062EB73E01DC087E18093430568E673E0CC
:1033200017C088E18093430567E573E011C089E128
:103330008093430563E473E00BC08AE18093430507
:103340006EE273E005C08BE18093430566E073E0B5
:1033500080EE95E00E94462A2FC06CEE72E080EE6F
:1033600095E00E94462A8091AB0591E01DC066ED74
:1033700072E080EE95E00E94462A8091AB0592E0D3
:1033800013C061EC72E080EE95E00E94462A8091C5
:10339000AB0594E009C066EA72E080EE95E00E9419
:1033A000462A8091AB0598E089278093AB058FEF83
:1033B000809343050E94021080EE95E00E946C2BE2
:1033C000892B09F45BC180EE95E00E94992BF4CF24
:1033D0000E940111882309F451C18091DD048111FB
:1033E00004C08FEF8093430541C140E050E060E0AE
:1033F00070E08EED94E00E94B32E40914305042FBF
:10340000112707FD1095212F312FF8013197EB314E
:10341000F10508F01BC1E255FF4F0C943C2E5527D7
:1034200047FD50952091460530E0241735070CF4F0
:103430000DC18B019C010150110921093109003294
:1034400011052105310558F0C0904705E9E4F5E084
:10345000F12CD12CA8E2EA2E415051090FC0FA01FB
:10346000E356FA4F61506083D9C0DF0111972C9168
:1034700030E02417350729F0F3943296FC10F5CF8D
:10348000CBC00E2D10E020E030E00617170728070C
:10349000390741F42081DA01A356BA4F11962C93D3
:1034A000DD24D394E394E8CF6F3F71058105910546
:1034B00011F008F0CBC06093B505B0C06F3F710547
:1034C0008105910511F008F0C1C06093B605A6C052
:1034D0006F3F71058105910511F008F0B7C0609349
:1034E000B7059CC02091DE0420622037E9F440E05B
:1034F00050E060E070E08FED94E00E94B32E9B01FD
:10350000AC01DC01CB010197A109B1090897A10524
:10351000B10508F0AEC0A4EDB0E30E948D2D6A5E47
:103520007C4A8A46954E24C02636E9F440E050E0B5
:1035300060E070E08FED94E00E94B32E9B01AC013F
:10354000DC01CB010197A109B1090797A105B105DC
:1035500008F08FC0A8EAB1E60E948D2D645E7C431E
:103560008E46944E05C0611571058105910579F06F
:103570008B019C01005C1D49284535430130FAE56B
:103580001F07F2E62F07F2E03F0708F05FC06093E5
:10359000AD057093AE058093AF059093B0053EC026
:1035A0006F3F71058105910511F008F04FC06093E0
:1035B000B10534C08B019C01015011092109310969
:1035C0000F3F11052105310508F040C06093B20599
:1035D00025C08B019C01045C1940210931090D347F
:1035E0004DE114072105310528F47093B40560936B
:1035F000B30514C0611571058105910521F48FEFA4
:103600008093AC050BC06134710581059105F0F420
:1036100061506093AC0502C0DD20C1F08091DC04F4
:1036200081111AC080917D0590917E05A0917F0542
:10363000B09180050196A11DB11D80937D059093E9
:103640007E05A0937F05B093800506C060E772E019
:1036500080EE95E00E94582A0E94F7108FEF809329
:1036600043056AE080EE95E00E946A2A0E940210FB
:1036700005C061E070E080E090E07ACF6C96E8E011
:103680000C942B2E6AE572E080EE95E00E94462AAB
:1036900062E472E080EE95E00E94462A80EE95E0BA
:1036A0000E946C2B892B31F080EE95E00E94992BC3
:1036B0000E94BA180E949217823029F0833051F488
:1036C0006DE072E002C064E272E080EE95E00E947C
:1036D000462A08958FEF809343051092DC040E94E0
:1036E0000210809143058E3F69F080EE95E00E94C4
:1036F0006C2B892BB1F380EE95E00E94992B0E94F0
:10370000BA18EFCF08950F931F93109143051F3FF1
:1037100009F0D2C0893409F457C000F5883309F4A0
:1037200069C058F4803309F477C008F061C08B3168
:1037300009F440C08132B1F1B9C0813409F487C0C5
:1037400030F4893309F466C0803461F1AFC082344B
:1037500009F48EC0863409F448C0A8C0823609F442
:1037600087C078F4883531F128F48235C1F183358A
:10377000E1F09CC08A3509F494C0813609F467C031
:1037800095C0823761F128F4863679F18936E1F007
:103790008DC0883779F08A3709F483C0833709F000
:1037A00085C003C061E172E015C00E94320D6EE871
:1037B00072E004C00E943B0D68EA72E080EE95E082
:1037C0000E94582A8EEF70C00E947A060E94BF069F
:1037D00067EC72E080EE95E00E94582A67C081E0B5
:1037E0000E94DF0660EE72E0F5CF0E94AC105EC072
:1037F00080535AC06AEF71E080EE95E00E94462A3D
:1038000090919C0588E0890F8871977E892B809321
:103810009C051AC089E048C067EE71E080EE95E033
:103820000E94462A8091BD059091BE05A091BF05DA
:10383000B091C00520E182278093BD059093BE051D
:10384000A093BF05B093C005109343052FC061ED51
:1038500071E080EE95E00E94462A8091BD0590912E
:10386000BE05A091BF05B091C00540E4842710C0FB
:1038700060EC71E080EE95E00E94462A8091BD05E3
:103880009091BE05A091BF05B091C00520E28227AE
:103890008093BD059093BE05A093BF05B093C0056E
:1038A00002C00E94421B8FEF809343058091430525
:1038B0008E3F09F0D4C0DDC00E940111882309F4B5
:1038C000D8C08091DD04811104C08FEF809343053F
:1038D000C6C040E050E060E070E08EED94E00E94F1
:1038E000B32E00914305112707FD1095212F312F8D
:1038F000F8013197E930F10508F0B4C0E753FF4F04
:103900000C943C2E8B019C01015C1D4928453543DC
:103910000F3F19452246324008F0A4C06093790554
:1039200070937A0580937B0590937C0577C06093B4
:103930007D0570937E0580937F059093800581E0DF
:103940008093DC046BC0683071058105910508F037
:1039500089C06093810562C08B019C0101501109EF
:10396000210931090A3011052105310508F07AC015
:103970006093820553C061EB71E08EED94E00E948C
:10398000ED2F10E0009799F00E94C72F009779F073
:10399000183130F4E12FF0E0EC58FA4F87871F5FC1
:1039A00061EB71E080E090E00E94ED2FEBCF1831E9
:1039B000A8F5E12FF0E0EC58FA4F17861F5FF7CF1C
:1039C000653071058105910508F04CC060939B0539
:1039D00025C08B019C0101501109210931090630D4
:1039E000110521053105F0F520919C05287F262B36
:1039F00020939C0513C08B019C01015011092109E2
:103A000031090115124C2140310560F560937505AF
:103A10007093760580937705909378058091DC0408
:103A2000811113C080917D0590917E05A0917F0545
:103A3000B09180050196A11DB11D80937D059093E5
:103A40007E05A0937F05B09380050E94F7108FEF4D
:103A5000809343056AE080EE95E00E946A2A0E9406
:103A6000351807C060E772E080EE95E00E94582AA2
:103A7000ECCF1F910F9108958FEF80934305109223
:103A8000DC040E943518809143058E3F69F080EE7A
:103A900095E00E946C2B892BB1F380EE95E00E949B
:103AA000992B0E94831BEFCF6AE070E080E090E0EA
:103AB0000E948F2880EE95E00E946C2B892B29F0C4
:103AC00080EE95E00E94992BF5CF0895CF93C82FF3
:103AD000682F80EE95E00E94C62B909168059C2788
:103AE00090936805CF910895A1E0B0E0EAE7FDE189
:103AF0000C94152E99830E94661D9981892F0E942E
:103B0000661D2196E2E00C94312E1F93CF93DF9334
:103B1000182FEB011092680565EB70E080EE95E0E0
:103B20000E94590662E670E080EE95E00E94590618
:103B3000812F0E94661DCE010E94741DDF91CF91DE
:103B40001F9108956091680580EE95E00E94C62B54
:103B50000895A1E2B0E0EFEAFDE10C94112E7B01A3
:103B60008A018C3009F453C108F040C0863009F452
:103B7000BCC018F5833009F491C070F4813009F4A9
:103B800072C0823009F048C26BE170E082E00E94AE
:103B9000851D0DE915E078C0843009F487C08530B3
:103BA00009F03AC26091470570E0660F771F85E023
:103BB0000E94851D08E415E086C0893009F4A7C07D
:103BC00070F4873009F49BC0883009F025C261E0A9
:103BD00070E088E00E94851D8091D20523C28A3062
:103BE00009F4CAC08B3009F4F2C016C28A3609F44F
:103BF00075C1D8F4873609F43AC138F4853609F42A
:103C00000EC1863609F41FC107C2883609F437C1D0
:103C1000893609F001C261E070E089E60E94851DE5
:103C20000E947A060E94BF06F5C18D3609F4D4C100
:103C300038F48B3609F491C18C3609F49AC1ECC181
:103C40008E3609F4DCC1873C09F0E6C161E070E022
:103C500087EC0E94851D81E00E94661D0E94A21DC6
:103C600010926905E3C169E270E081E00E94851D60
:103C700004E715E0F80181918F010E94661DF5E0CF
:103C80000D391F07B9F7D0C1F80181918F010E944A
:103C9000661DF5E0083B1F07B9F7C6C161E070E09B
:103CA00083E00E94851D0E949217BCC161E070E014
:103CB00084E00E94851D81E00E94661D0E94A21D75
:103CC0000E94C515B3C18091470590E0880F991FE8
:103CD0009801285435402817390708F0A5C1F80184
:103CE00081918F010E94661DEECF62E070E086E058
:103CF0000E94851D80E893E00E94741D95C161E0DB
:103D000070E087E00E94851D809146058BC186E6A4
:103D1000898361E0CE0101960E94DB0B0E94590B62
:103D200083E08093710568EC70E080E090E00E9491
:103D30008F28809171058430D9F48FE70E9477092C
:103D40000E948A098983863469F460E270E089E020
:103D50000E94851D10E20E948A090E94661D115072
:103D6000D1F762C161E070E089E00E94851D52C117
:103D700061E070E089E053C169E170E08AE00E948F
:103D8000851D82E08093B805209170058091BD0566
:103D90009091BE05A091BF05B091C005222311F0FE
:103DA000806801C08F778093BD059093BE05A09376
:103DB000BF05B093C00508EB15E0F80181918F01B4
:103DC0000E94661DF5E0013D1F07B9F72DC161E2B4
:103DD00070E08BE00E94851D8091A8048F3F39F030
:103DE0008091A80491E0980F9093A80402C080915C
:103DF000A8040E94661D10E0812F0E94A7150E9452
:103E000009090E94741D1F5F1031B1F70DC161E0F7
:103E100070E08CE00E94851D8091D10503C161E0B6
:103E200070E085E60E94851D89E2E816F10409F03C
:103E3000F8C0D801E4E7F5E08D91819385E0ED3994
:103E4000F807D1F7E7C061E070E086E60E94851DC3
:103E5000EBE1EE16F10409F0E4C0D801EDE9F5E07C
:103E60008D91819385E0E83BF807D1F7D3C061E0FD
:103E700070E087E60E94851D0E94320DCBC061E094
:103E800070E088E60E94851D85E789838BE1EDE976
:103E9000F5E0DE01129601900D928A95E1F76CE152
:103EA000CE0101960E94DB0B0E94590B83E08093A8
:103EB000710560E273E080E090E00E948F288091BD
:103EC0007105843009F0ADC08FE70E9477090E9428
:103ED0008A098983853509F0A4C09CC061E070E03F
:103EE0008AE60E94851D89E6898361E0CE010196FC
:103EF0000E94DB0B0E94590B83E08093710560E206
:103F000073E080E090E00E948F28809171058430FA
:103F100009F087C08FE70E9477090E948A09898388
:103F20008E010E5F1F4F7E01EDE1EE0EF11C0E942F
:103F30008A09F80181938F01EE15FF05C1F78BE126
:103F4000FE013296ADE9B5E001900D928A95E1F758
:103F50008981893409F065C05DC061E070E08BE65D
:103F60000E94851DF80180818093D2050E943B0D3F
:103F700051C061E070E08CE60E94851DF0E2EF1612
:103F8000F10461F487E6898380E2F801DE0112968C
:103F900001900D928A95E1F761E203C087E489837D
:103FA00061E0CE0101960E94DB0B0E94590B83E079
:103FB000809371056CE474E080E090E00E948F28AB
:103FC00080917105843069F58FE70E9477090E941E
:103FD0008A09873431F51EC061E070E08DE60E94E9
:103FE000851D89E1E816F104E1F4D801E8EBF5E07C
:103FF0008D91819385E0E13DF807D1F70BC061E039
:1040000070E08EE60E94851DF80180818093D105C5
:104010000E941B0D81E006C061E070E08AEC0E9406
:10402000851D80E00E94661D0E94A21DA196E6E00B
:104030000C942D2EA0E0B0E0E0E2F0E20C940F2E04
:10404000CAECD3E014E606E035E0F32E44E0E42EBB
:1040500053E0D52E62E0C62E80EE95E00E946C2BD8
:10406000892B09F49BC080EE95E00E94992B282FA4
:10407000809335044091340450E04730510560F797
:10408000FA01EE52FF4F0C943C2E853B29F781E05C
:1040900080933404E1CF823609F07DC0C0923404AD
:1040A000DBCF8093330480933204D0923404D4CF96
:1040B0009C013327309331042093300490913204D3
:1040C000982790933204E0923404C6CF382F2227E9
:1040D0004091300450913104242B352B309331041E
:1040E0002093300490913204982790933204F092F8
:1040F00034042536310508F4AFCF61E070E08CEC74
:104100000E94851D81E00E94661D0E94A21D43C081
:1041100020912E0430912F04F901E653FC4F808347
:1041200090913204982790933204C901019690939C
:104130002F0480932E042091300430913104821793
:10414000930708F489CF0093340486CF809132041A
:1041500082130BC060912E0470912F044AEC53E03F
:10416000809133040E94A91D0DC062E070E08BECC9
:104170000E94851D809133040E94661D8091680510
:104180000E94661DFE01812F11928A95E9F7109217
:104190002F0410922E04109234045ECFCDB7DEB7F8
:1041A000E8E00C942B2E81E08093690580916905ED
:1041B000882349F080EE95E00E946C2B892BB1F3A7
:1041C0000E941A20F3CF0895AAE2B0E0EAEEF0E2EE
:1041D0000C940D2E0E9460286B017C0181E00E94EE
:1041E0007E0A80EE95E00E946C2B892B29F080EEF0
:1041F00095E00E94992BF5CF2D9811E072E6B72E2D
:10420000E9E2AE2E03E00E9460286C197D098E0958
:104210009F09693C710581059105D0F11123C1F118
:104220000E9460286B017C012C9A80ED97E00E942F
:10423000A807B982E4E7F5E0DE0112968A2D019025
:104240000D928A95E1F76AE2CE0101960E94DB0B9E
:104250002C9880E090E00E94A807009371050E94CE
:10426000590B62E370E080E090E00E948F2880911B
:104270007105843061F4009371058FE70E9477091E
:104280000E948A0911E0823419F410E001C011E0A3
:104290008BE00E948529892B81F411E00EC02D9AB4
:1042A0002C9A80EE95E00E94992B8D309105A9F013
:1042B0005CF40A9791F02D982C9880EE95E00E947E
:1042C0006C2B892B61F79FCF8332910579F0823473
:1042D000910589F70E94D320EECF62EB71E080EE6A
:1042E00095E00E94462A0E943C1DE5CF0E94C5151C
:1042F000E2CF8F929F92AF92BF92CF92DF92EF92D6
:10430000FF921F93CF93DF938BE00E948529892B27
:1043100009F089C068EC70E080E090E00E948F288E
:1043200080E090E00E94A8070E9460284B015C0199
:104330006B017C0180ECC80E82E1D81EE11CF11CEF
:104340000E9460286C157D058E059F0530F48BE07A
:104350000E948529892BA1F364C08BE00E948529E6
:10436000892B09F05EC080ED97E00E94A8070E94AB
:1043700060286B017C01D0E0C1E088E4880E86E211
:10438000981EA11CB11C11E08BE00E948529892B8D
:1043900021F58C149D04AE04BF0430F480ED97E049
:1043A0000E94A807D1E0F0CF0E9460286C197D0917
:1043B0008E099F09693C71058105910528F30E94CA
:1043C00060286B017C01C12719F080ED97E002C0E5
:1043D00080E090E00E94A807D7CF80E090E00E94A4
:1043E000A807DD23B9F08091D10590E0019665E042
:1043F00070E00E94B02D8093D1050E941B0D0E9499
:104400009C130E943B0D64EF71E080E090E00E94FD
:104410008F2809C080E00E94DF060E94B3110E942D
:10442000320D0E94E420DF91CF911F91FF90EF9019
:10443000DF90CF90BF90AF909F908F900895CF92D4
:10444000DF92EF92FF9280E00E94DA070E94B107AC
:1044500061E08DE00E94192961E08CE00E94192939
:1044600060E08BE00E94192960E083E00E94192936
:1044700061E083E00E94522961E08EE00E941929E8
:1044800060E08EE00E9452290E949F0740E052ECBB
:1044900061E070E080EE95E00E94B42C0E949C13D5
:1044A0000E943B0D0E9485138FEF8093A8040E9409
:1044B000C60778940E9460286B017C018091A80453
:1044C0008F3F59F40E9460286C197D098E099F095D
:1044D000603D77408105910588F380ED97E00E946B
:1044E000A80761E08BE00E9452292D9A80EE95E0AA
:1044F0000E946C2B892B29F080EE95E00E94992B6D
:10450000F5CF6DEF72E080EE95E00E94272A80E8FB
:1045100093E00E94300C64E173E080EE95E00E942D
:10452000272A4AE050E062E070E080EE95E00E94C9
:10453000F72A62E370E080E090E00E948F2880EE2E
:1045400095E00E946C2B04970CF180EE95E00E94A0
:10455000992B82349105D1F480EE95E00E94992B3D
:104560008E34910599F480EE95E00E94992B843465
:10457000910561F480EE95E00E94992B819731F4CA
:1045800080E090E00E94A8070E94E4204091750519
:10459000509176056091770570917805DB01CA012D
:1045A0000197A109B1090497A105B10568F44093E9
:1045B000A704433029F440EA56E861E070E004C003
:1045C00040E052EC61E070E080EE95E00E94B42C97
:1045D0000E9479212D9880E090E00E94A8070E9417
:1045E00085131092C3048091BD0583FF11C0809193
:1045F0008905882351F080919005882331F08091BE
:104600009705882311F087E001C085E08093C304FB
:1046100080E00E947E0A8091C4040E94B2090E9438
:10462000590B10923F0410923E0410923D04F12C5D
:104630008091D2058F15B0F062E370E080E090E0E9
:104640000E948F2880ED97E00E94A80762E370E047
:1046500080E090E00E948F2880E090E00E94A80710
:10466000F394E6CF80919C0584FF08C0982F987141
:1046700081E0983109F080E00E946F118FE00E9484
:10468000DA07FF90EF90DF90CF900895EF92FF92BE
:104690000F931F93CF93DF938C016EE770E080EE52
:1046A00095E00E945906E801F12CF0E2EF2E8E0110
:1046B00088818D57823048F46DE770E080EE95E098
:1046C0000E94590688818E2588832196F801608191
:1046D00080EE95E00E94C62BF394F9E0FF12E7CF3D
:1046E0006EE770E080EE95E00E945906CDB7DEB728
:1046F000E6E00C942D2EA9E0B0E0E1E8F3E20C94A2
:10470000152E9091C50491110EC09EEF99838A8356
:104710006B8350E0559547954C832D8319861886F9
:104720001F821E822EC04091CA04842F90E0B4E004
:1047300095958795BA95E1F7242F2F7030E0821771
:10474000930719F18DEF89831B82FE01349650E0A7
:10475000842F90E0A4E095958795AA95E1F7242F02
:104760002F7030E08217930749F0DC01A553BB4F4F
:104770008C918193405F5F5F563051F74093CA043C
:104780005A83CE0101960E9446238091C50490E091
:10479000019666E070E00E94B02D8093C5042996D2
:1047A000E2E00C94312EA0E0B0E0E9EDF3E20C94ED
:1047B0000E2E6C016EE770E080EE95E00E945906C7
:1047C0008601E12CF12CC0E0D0E030E2B32EF801FC
:1047D000608183E8860F823078F46DE770E080EEC8
:1047E00095E00E945906F80160816B2570E080EE2B
:1047F00095E00E94590604C080EE95E00E94C62B09
:10480000E114F10459F0F80180819E01280F311D57
:10481000C901C92FDD27C80FD91FDD273FEFE31AD4
:10482000F30A89E0E816F10459F028E0E216F104F1
:1048300021F48C2F8095F60180870F5F1F4FC7CF23
:10484000CDB7DEB7E9E00C942A2EA9E0B0E0EBE2A8
:10485000F4E20C94152EE82F362F8091C50490E0D9
:10486000019664E270E00E94B02D8093C50458E97F
:10487000598350E15A83813089F048F08230B9F091
:104880008330D9F48B8381EF8C833D8319C085E01D
:104890008B8381EF8C832F5F2D8312C08B8381EFFD
:1048A0008C8384E6489FA00111245D8309C084E0C5
:1048B0008B8381EF8C83ED8303C00E94AC1104C015
:1048C000CE0101960E94D3232996E2E00C94312E6A
:1048D000A2E0B0E0EEE6F4E20C940A2E182F762E59
:1048E0002A8349830E946C286B017C018091DB0440
:1048F0008090C6049090C704A090C804B090C904EA
:104900002A8149818823C1F0D701C60188199909F4
:10491000AA09BB094C015D0191EE89169EE2990638
:10492000A104B10420F1241708F4422F202F672D91
:10493000812F0E94252413C0D701C6018819990927
:10494000AA09BB094C015D0191E3891695E7990617
:10495000A104B10460F0672D812F0E947B23C092D7
:10496000C604D092C704E092C804F092C90422960B
:10497000EDE00C94262EA2E2B0E0E1ECF4E20C941F
:104980000B2E8CE00E94990981110DC06CE173E03F
:1049900080EE95E00E94582A2D9A80E00E947E0ABF
:1049A0000E94590B2D9880EE95E00E946C2B892B6C
:1049B00001F180EE95E00E94992B9091A704992334
:1049C00019F00E94AF13EFCF40913E0450E09A01DE
:1049D0002F5F3F4F2F71332760913F0470E0261700
:1049E000370709F3FA01E75BFB4F808320933E040E
:1049F000DACF80917105843009F086C00E946C285E
:104A0000611571058105910549F06093B5047093B6
:104A1000B6048093B7049093B8040CC081E090E092
:104A2000A0E0B0E08093B5049093B604A093B704DF
:104A3000B093B8048091AB049091AC0481609093E2
:104A4000AC048093AB0483E0809371058FE70E94F0
:104A5000770909E614E00E948A09F80181938F0121
:104A6000F4E002371F07B9F72091720480916904BE
:104A7000982F922796FF3BC090E492279093720460
:104A8000982F98739833F1F410E0212F30E0809143
:104A90006904877090E0821793074CF11F5F2091A3
:104AA0009C05812F90E0FC01E759FB4F24FF04C0D7
:104AB00080810E948E11E9CF608180EE95E00E9496
:104AC000C62BE3CF8F7399F480916A048093B4046A
:104AD00080916B048093B20480916C048093B10444
:104AE00080916F0490E09093AA048093A904809130
:104AF0003D04813019F482E080933D0480913D04AF
:104B0000833011F410923D040E946C286B017C01EB
:104B10008091AD049091AE04A091AF04B091B00427
:104B20000097A105B105C9F0A7019601281B390B13
:104B30004A0B5B0BDA01C901883B9B40A105B1051B
:104B400060F00E94C8098093B3041092AD041092E3
:104B5000AE041092AF041092B0048091B904909109
:104B6000BA04A091BB04B091BC0446015701881A55
:104B7000990AAA0ABB0A84E795E00E94F407861600
:104B80009706A806B90608F4A8C0C092B904D09246
:104B9000BA04E092BB04F092BC040E9457068091D4
:104BA000A8048830A0F08091BD059091BE05A09129
:104BB000BF05B091C0056CE1B695A795979587950F
:104BC0006A95D1F7892B8A2B8B2B09F0A4C1809190
:104BD000A8048F5F8093A8048091B5049091B604D7
:104BE000A091B704B091B8040097A105B105F1F008
:104BF000C81AD90AEA0AFB0A84E795E00E94F4077A
:104C00006C157D058E059F0508F006C18091BD05D8
:104C100084FD04C080ED97E00E94A8071092B504BF
:104C20001092B6041092B7041092B80490917204D6
:104C3000907C9093720450913E0480913F042091A7
:104C40003D04581709F405C1223009F002C19058FB
:104C500090937204E0919C05E770F0E0E658FC4FF9
:104C60006081693008F0DDC0615040E04613DBC070
:104C700080933F0487E3840F90917204892B809383
:104C800072044093400483E080933D042C9A809109
:104C900081059091C30491112FC10E94790A8091DE
:104CA000C4040E94B209E0919C05E770F0E0E65868
:104CB000FC4F608182E794E00E94940BE091C40471
:104CC000EF5FE093C404E83109F422C1F0E0EC584E
:104CD000FA4F8785882309F41BC10E94030C813099
:104CE00069F580919C05887149F18091AB049091A0
:104CF000AC04880F991F9093AC048093AB0483E0BD
:104D0000809371050E94590B0E946C286093AD043A
:104D10007093AE048093AF049093B004672B682B1C
:104D2000692B61F481E090E0A0E0B0E08093AD04F5
:104D30009093AE04A093AF04B093B00480919C050F
:104D400084FF1FC08091AB049091AC048E7F0E94C1
:104D50002A09182F6091A9048091B4040E94A51318
:104D6000482F612F8091B30449A30E94A51300919D
:104D7000D205282F49A16091B1048091B2040E940C
:104D800068242C988091C1048130C1F018F08230E1
:104D9000B1F1CEC08BE00E948529892B09F0C8C0F3
:104DA00081E08093C1040E9460286093BD047093E9
:104DB000BE048093BF049093C004BAC08BE00E94ED
:104DC0008529892B31F50E946028C090BD04D090C0
:104DD000BE04E090BF04F090C0046C197D098E09F8
:104DE0009F09693E73408105910508F4A1C082E0E6
:104DF0008093C10480ED97E00E94A80799C08BE0E2
:104E00000E948529892B09F493C080E090E00E94DC
:104E1000A8071092C1048CC080E090E00E94A8070F
:104E200005CF68E022CF851709F422CF4F5F242FEA
:104E300030E090E0F901EE58FB4FDC01A75BBB4F7F
:104E40007C917083F901E05CFB4F708301968F7158
:104E50000DCF2430B1F42091400481E494E0A3E725
:104E6000B4E0FC013E2F381B321718F431913D930A
:104E7000F9CF87E3820F90917204892B809372049B
:104E800002CF8091C104823069F4916090937204E2
:104E90002D9A51ECE52E55E0F52E8E010F5F1F4F38
:104EA000B80110C02D9880913D04811103C081E0AC
:104EB00080933D0480913D04833059F784E08093D2
:104EC0003D04E7CFF70181917F0169A37AA30E9496
:104ED000A715F801819391938F0169A17AA1F1ED52
:104EE000EF16F5E0FF0671F780919C0543E754E06B
:104EF00087700E947908CACE882309F4CECE20910B
:104F0000C20431E0320F3093C2042913C6CE0CC064
:104F10001092C404E2CE8091A804883009F42D9A3E
:104F200089E08093A804D9CE1092C2048150B5CEF6
:104F3000A296ECE00C94272E8230E8F4E82FF0E003
:104F4000EE0FFF1FED52FA4F71836083813041F005
:104F5000809169008C7F842B80936900E89A089582
:104F600080916900440F551F440F551F837F842B88
:104F700080936900E99A08951F920F920FB60F92DD
:104F800011242F933F934F935F936F937F938F934E
:104F90009F93AF93BF93EF93FF938091D30590912D
:104FA000D405892B29F0E091D305F091D40509951A
:104FB000FF91EF91BF91AF919F918F917F916F91F1
:104FC0005F914F913F912F910F900FBE0F901F90C7
:104FD00018951F920F920FB60F9211242F933F93A3
:104FE0004F935F936F937F938F939F93AF93BF93F1
:104FF000EF93FF938091D5059091D605892B29F0E9
:10500000E091D505F091D6050995FF91EF91BF91FB
:10501000AF919F918F917F916F915F914F913F9150
:105020002F910F900FBE0F901F9018951F920F9207
:105030000FB60F9211242F933F938F939F93AF93AB
:10504000BF938091D8059091D905A091DA05B091D0
:10505000DB053091D70523E0230F2D3720F401968F
:10506000A11DB11D05C026E8230F0296A11DB11D8B
:105070002093D7058093D8059093D905A093DA059E
:10508000B093DB058091DC059091DD05A091DE05F4
:10509000B091DF050196A11DB11D8093DC059093B1
:1050A000DD05A093DE05B093DF05BF91AF919F9121
:1050B0008F913F912F910F900FBE0F901F901895D9
:1050C0002FB7F8946091D8057091D9058091DA05D1
:1050D0009091DB052FBF08953FB7F8948091DC05D0
:1050E0009091DD05A091DE05B091DF0526B5A89B66
:1050F00005C02F3F19F00196A11DB11D3FBF6627C6
:10510000782F892F9A2F620F711D811D911D42E00A
:10511000660F771F881F991F4A95D1F70895CF9280
:10512000DF92EF92FF92CF93DF936B017C010E949D
:105130006C28EB01C114D104E104F10479F00E9460
:105140006C286C1B7D0B683E7340A0F381E0C81A8D
:10515000D108E108F108C851DC4FECCFDF91CF91C5
:10516000FF90EF90DF90CF900895789484B582609F
:1051700084BD84B5816084BD85B5826085BD85B5FB
:10518000816085BDEEE6F0E0808181608083E1E8AA
:10519000F0E01082808182608083808181608083E2
:1051A000E0E8F0E0808181608083E1EBF0E08081E5
:1051B00084608083E0EBF0E0808181608083EAE7B7
:1051C000F0E0808184608083808182608083808140
:1051D000816080838081806880831092C1000895FF
:1051E000833081F028F4813099F08230A1F0089565
:1051F0008630A9F08730B9F08430D1F480918000F6
:105200008F7D03C0809180008F7780938000089508
:1052100084B58F7702C084B58F7D84BD0895809159
:10522000B0008F7703C08091B0008F7D8093B00075
:105230000895CF93DF9390E0FC01ED50F44F24915B
:10524000FC01E95FF34F8491882349F190E0880FD6
:10525000991FFC01E15DF34FA591B4918B5D934FD4
:10526000FC01C591D4919FB7611108C0F8948C914D
:10527000209582238C93888182230AC0623051F466
:10528000F8948C91322F309583238C938881822BD4
:10529000888304C0F8948C91822B8C939FBFDF91FC
:1052A000CF910895A1E0B0E0E8E5F9E20C94132E67
:1052B000282F30E0F901E152F44F8491F901ED50CB
:1052C000F44F1491F901E95FF34F04910023C9F001
:1052D000882321F069830E94F0286981E02FF0E0A3
:1052E000EE0FFF1FEB5DF34FA591B4919FB7F894BC
:1052F0008C91611103C01095812301C0812B8C9387
:105300009FBF2196E4E00C942F2ECF93DF93282F9C
:1053100030E0F901E152F44F8491F901ED50F44F7E
:10532000D491F901E95FF34FC491CC2391F081113D
:105330000E94F028EC2FF0E0EE0FFF1FE55EF34F28
:10534000A591B4912C912D2381E090E021F480E08F
:1053500002C080E090E0DF91CF9108958E3008F098
:105360008E50877020919D0190E4299F9001112417
:10537000822B80937C0080917A00806480937A00F5
:1053800080917A0086FDFCCF809178002091790091
:1053900090E0922B0895A0E0B0E0E1EDF9E20C94EA
:1053A0000F2E6C017A01EB01E60EF71E00E010E013
:1053B000CE15DF0561F06991D601ED91FC91019068
:1053C000F081E02DC6010995080F191FF1CFC80122
:1053D000CDB7DEB7E8E00C942B2E6115710589F08E
:1053E000DB010D900020E9F7AD0141505109461B4A
:1053F000570BDC01ED91FC910280F381E02D0995C2
:10540000089580E090E00895EF92FF920F931F932C
:10541000CF93DF938C01FB01C0E0D0E064917F016A
:105420008FEFE81AF80A662361F0D801ED91FC913C
:105430000190F081E02DC8010995C80FD91FF7012F
:10544000EDCFCE01CDB7DEB7E6E00C942D2E0E9455
:10545000ED290895DC01ED91FC910190F081E02DA2
:10546000099508950F931F93CF93DF93EC016DE09F
:105470000E942A2A8C016AE0CE010E942A2A800F0B
:10548000911FDF91CF911F910F9108950F931F935B
:10549000CF93DF93EC010E94042A8C01CE010E947D
:1054A000322A800F911FDF91CF911F910F910895A4
:1054B0000F931F93CF93DF93EC010E94ED298C0192
:1054C000CE010E94322A800F911FDF91CF911F9150
:1054D0000F9108950F931F93CF93DF93EC010E94D8
:1054E0002A2A8C01CE010E94322A800F911FDF915F
:1054F000CF911F910F910895A1E2B0E0E2E8FAE2A6
:105500000C940B2E7C01C42EE52FCB01D22E19A2B8
:1055100021E02D1510F02AE0D22E8E010F5D1F4FD5
:105520008D2C912CA12CB12C6C2D7E2FA5019401DA
:105530000E94C42D8C2DD29E801911240150110976
:105540008A3010F4805D01C0895CF80180832115E8
:1055500031054105510521F0C22EE32FCA01E4CFE8
:10556000B801C7010E94ED29A196ECE00C94272E0A
:10557000A0E0B0E0EEEBFAE20C940F2EEC016A0131
:105580007B012115310541F4E881F9810190F08119
:10559000E02D642F09951DC02A303105A9F477FF4D
:1055A00012C06DE20E942A2A8C0144275527BA01B5
:1055B0004C195D096E097F092AE0CE010E947C2A00
:1055C000800F911F06C02AE0B701A601CE010E94FC
:1055D0007C2ACDB7DEB7E8E00C942B2E9A01AB0104
:1055E000662757FD6095762F0E94B82A08950F937D
:1055F0001F93CF93DF93EC019A01AB01662757FD10
:105600006095762F0E94B82A8C01CE010E94322A22
:10561000800F911FDF91CF911F910F910895211558
:10562000310549F4DC01ED91FC910190F081E02D10
:10563000642F099508950E947C2A08959A01462FA7
:1056400050E060E070E00E940F2B08959A01AB01DA
:1056500060E070E00E940F2B08950F931F93CF938B
:10566000DF93EC010E940F2B8C01CE010E94322AA5
:10567000800F911FDF91CF911F910F9108950F938C
:105680001F93CF93DF93EC019A01AB0160E070E0D0
:105690000E940F2B8C01CE010E94322A800F911F95
:1056A000DF91CF911F910F9108950F931F93CF9387
:1056B000DF93EC019A01462F50E060E070E00E9419
:1056C0000F2B8C01CE010E94322A800F911FDF9197
:1056D000CF911F910F910895FC0124853585F90123
:1056E000E05CFF4F80819181F901EE5BFF4F2081EB
:1056F0003181821B930B8F7399270895FC01848558
:105700009585FC01E05CFF4F40815181FC01EE5B1F
:10571000FF4F208131814217530741F00190F08102
:10572000E02DE80FF91F808190E008958FEF9FEF43
:105730000895FC0184859585FC01E05CFF4F408164
:105740005181FC01EE5BFF4F2081318142175307ED
:1057500079F0A081B181A80FB91F8C91208131818E
:105760002F5F3F4F2F7333273183208390E00895BD
:105770008FEF9FEF0895FC0181A1882329F0A48970
:10578000B5898C9186FFFBCF11A20895CF93DF934B
:10579000FC0126853785D901A05CBF4F8D919C9176
:1057A000119701968F739927E901CE5BDF4F4881EE
:1057B000598184179507D9F30D90BC91A02DA20FA4
:1057C000B31F6C93A685B785A05CBF4F11969C93C1
:1057D0008E93A689B7892C9181E090E0078C02C056
:1057E000880F991F0A94E2F7282B2C9381E081A35C
:1057F0000488F589E02D80818064808381E090E0D9
:10580000DF91CF91089508951F920F920FB60F92D6
:1058100011242F933F934F938F939F93EF93FF9375
:105820008091C00082FD1CC04091C6008091860618
:105830009091870601968F73992720918806309161
:1058400089068217930771F0E0918606F09187062A
:10585000EA5BF94F4083909387068093860602C0E7
:105860008091C600FF91EF919F918F914F913F9151
:105870002F910F900FBE0F901F90189580EE95E01E
:105880000E946C2B892B11F00E94032C08951F920B
:105890000F920FB60F9211242F933F938F939F93E4
:1058A000EF93FF9320914206309143068091440686
:1058B000909145062817390731F48091C1008F7DFA
:1058C0008093C10014C0E0914406F0914506EE5F5C
:1058D000F94F2081809144069091450601968F737F
:1058E000992790934506809344062093C600FF9124
:1058F000EF919F918F913F912F910F900FBE0F903D
:105900001F901895A0E0B0E0E8E8FCE20C940B2EA4
:10591000FC011382128288EE93E0A0E0B0E0848361
:105920009583A683B7838CEB93E0918380837587FF
:10593000648757874687318B208B138B028BF58AC0
:10594000E48AD78AC68AB18EA08E938E828E8F8586
:10595000848F8889858F8989868F8A89878F8B89AB
:1059600080A3ECE00C94272ECF92DF92EF92FF926F
:10597000CF93DF93EC016A017B01411581EE58075B
:1059800061057105F9F0EC89FD8981E090E008A0DE
:1059900002C0880F991F0A94E2F7808360E079E0E3
:1059A0008DE390E0A70196010E94C42D215031099A
:1059B000410951095695479537952795211580E15D
:1059C000380798F0EC89FD89108260E874E88EE170
:1059D00090E0A70196010E94C42D21503109410990
:1059E00051095695479537952795E889F989308368
:1059F000EA89FB89208319A2EE89FF89408181E031
:105A000090E09C010C8C02C0220F331F0A94E2F735
:105A1000422B4083EE89FF8940819C010D8C02C09E
:105A2000220F331F0A94E2F7422B4083EE89FF894D
:105A300040819C010E8C02C0220F331F0A94E2F7B2
:105A4000422B4083EE89FF8920810F8C02C0880F92
:105A5000991F0A94E2F7809582238083DF91CF918A
:105A6000FF90EF90DF90CF9008958F929F92AF922A
:105A7000BF92CF92DF92EF92FF920F931F9381E03C
:105A80008F9385E08F9387E08F9383E08F9384E0FB
:105A90008F93E6EC8E2E912CF2ECAF2EB12CA1EC74
:105AA000CA2ED12CB0ECEB2EF12C04EC10E025EC3E
:105AB00030E042E056E066E476E080EE95E00E9459
:105AC000822C0F900F900F900F900F901F910F91BD
:105AD000FF90EF90DF90CF90BF90AF909F908F900E
:105AE00008950E94B5280E941F22CEE3DCE20E94A6
:105AF000BB242097E1F30E943E2CF9CFA29FB00176
:105B0000B39FC001A39F700D811D1124911DB29FF1
:105B1000700D811D1124911D08950E947E2DA59F59
:105B2000900DB49F900DA49F800D911D1124089598
:105B3000B7FF0C948D2D0E948D2D821B930B089521
:105B4000DB018F939F930E948D2DBF91AF91A29FF8
:105B5000800D911DA39F900DB29F900D112408956B
:105B600097FB072E16F4009407D077FD09D00E940A
:105B7000422E07FC05D03EF4909581959F4F0895E5
:105B8000709561957F4F0895A1E21A2EAA1BBB1B49
:105B9000FD010DC0AA1FBB1FEE1FFF1FA217B307F9
:105BA000E407F50720F0A21BB30BE40BF50B661F0F
:105BB000771F881F991F1A9469F7609570958095D3
:105BC00090959B01AC01BD01CF010895052E97FB77
:105BD0001EF400940E94FD2D57FD07D00E94C42D95
:105BE00007FC03D04EF40C94FD2D50954095309554
:105BF00021953F4F4F4F5F4F089590958095709539
:105C000061957F4F8F4F9F4F08952F923F924F92F4
:105C10005F926F927F928F929F92AF92BF92CF923C
:105C2000DF92EF92FF920F931F93CF93DF93CDB745
:105C3000DEB7CA1BDB0B0FB6F894DEBF0FBECDBFBD
:105C400009942A88398848885F846E847D848C848E
:105C50009B84AA84B984C884DF80EE80FD800C8197
:105C60001B81AA81B981CE0FD11D0FB6F894DEBF7A
:105C70000FBECDBFED010895EE0FFF1F0590F4910B
:105C8000E02D0994AA1BBB1B51E107C0AA1FBB1F33
:105C9000A617B70710F0A61BB70B881F991F5A95B8
:105CA000A9F780959095BC01CD0108958F929F92A0
:105CB000AF92BF92CF92DF92EF92FF92CF93DF939A
:105CC000EC01688179818A819B816115710581056B
:105CD000910521F464E279ED8BE597E02DE133EF56
:105CE00041E050E00E94E62D49015A019B01AC01C0
:105CF000A7EAB1E40E948D2D6B017C01ACEEB4EFFC
:105D0000A50194010E949B2DC60ED71EE81EF91E08
:105D1000F7FE06C081E0C81AD108E10880E8F80A59
:105D2000C882D982EA82FB82C701B6019F77DF91E0
:105D3000CF91FF90EF90DF90CF90BF90AF909F906A
:105D40008F9008950E94562E089586E091E00E945B
:105D5000562E089560930601709307018093080101
:105D60009093090108952F923F925F926F927F92D4
:105D70008F929F92AF92BF92CF92DF92EF92FF925B
:105D80000F931F93CF93DF938B01EA016115710588
:105D900021F0DB018C9311969C93209739F09E01A2
:105DA000225031092332310508F0D8C07C01670147
:105DB000BFEFCB1ADB0A5601F7016080862D90E019
:105DC0000E94E52F892B11F07601F1CFFDE26F12D1
:105DD0000AC0570182E0A80EB11CD70111966C9041
:105DE000772473940BC0BBE26B1207C05701E2E04B
:105DF000AE0EB11CD70111966C90712CCE018F7E26
:105E0000892B89F4B0E36B1237C0F50180818F7D57
:105E10008835D1F46180F2E0AF0EB11C872D82602D
:105E2000782EC0E1D0E0CA30D10551F1C031D105A2
:105E300021F0C830D10599F409C0CC24CA94DC2CD7
:105E4000EC2CAFE0FA2E22C0209769F7C8E0D0E032
:105E5000CC24CA94DC2CEC2CFFE1FF2E17C06FEF92
:105E60007FEFCB019E01442737FD4095542F0E94C0
:105E7000C42D69017A010AC02097A9F6CAE0D0E0D2
:105E8000E9E9CE2EDC2CEC2CE9E1FE2EF50160E0F8
:105E900020E030E0A9014E01AA2497FCA094BA2C7E
:105EA0001F0170ED572E560CA9E0A51570F48FEB6D
:105EB000860D8A3118F499EC592E06C08FE9860DAB
:105EC0008A3148F589EA582E560C852D90E08C17BA
:105ED0009D070CF56F3FD9F0C216D306E406F50610
:105EE00098F0C501B4010E94A02D9B01AC01852D45
:105EF00090E0A0E0B0E0280F391F4A1F5B1F281771
:105F000039074A075B0710F46FEF01C061E0319673
:105F1000D1016C90C5CF0115110551F0662311F028
:105F2000319703C071FE04C03297D801ED93FC9302
:105F300070FE07C050954095309521953F4F4F4FCB
:105F40005F4F67FF10C082E290E090938B068093D2
:105F50008A066FEF7FEF8FEF9FEF07C060E070E082
:105F600080E090E002C0B901CA01DF91CF911F919A
:105F70000F91FF90EF90DF90CF90BF90AF909F90E8
:105F80008F907F906F905F903F902F900895FC01CD
:105F900088279927E89421912032E9F3293010F0DD
:105FA0002E30C8F32B3241F02D3239F4689404C0FE
:105FB0000E941930820F911D219120532A30C0F385
:105FC0001EF4909581959F4F0895911150C0803295
:105FD00019F089508550D0F7089548EC53E00E949D
:105FE000F22F0895FA01A191B081009719F410974A
:105FF000E1F0CD01DC01CD010D90002011F4C001D4
:1060000013C0FB012191222319F02015D9F7F3CFFA
:10601000FB012191201519F41E92119606C022232E
:10602000C1F70D900020A1F7D001FA01A193B08330
:1060300008957AE0979F902D879F802D910D1124D0
:106040000895F999FECF92BD81BDF89A992780B540
:106050000895262FF999FECF1FBA92BD81BD20BDAC
:106060000FB6F894FA9AF99A0FBE019608959927F7
:0860700088270895F894FFCF82
:1060780000008C06200001000000FF000200020062
:1060880002000200020002000200020002000200F8
:106098000200020002000200020002802500000542
:1060A800400AA1204EA50020244EA52C2330C01262
:1060B80000001A400AA1204EA5001B1E27522C23BF
:1060C800308025000005400AA1204EA50020244E5E
:1060D800A52C2330004B000006400AD0009D490043
:1060E8007B289D492C233000E1000005400A45012A
:1060F800D7DC03B81E0EBF00232E48E801008A40F3
:106108000A6001555502AD1E20000023C8015458ED
:106118002074696D656F75742100596573004E6F41
:10612800002C00386368004E2F41002C205B005D76
:106138002028002900486F70206368616E6E656CC6
:10614800200020402000456E746572696E672061EA
:1061580064617074697665206368616E6E656C2031
:1061680073656C656374696F6E2C207069636B6905
:106178006E673A007363616E6E6572206D6F646559
:10618800004E4F5420454E41424C45440053656EE5
:1061980064696E672073657474696E677320746FC1
:1061A8002052580A00526573657474696E672073CB
:1061B800657474696E6773206F6E2052580A0041C7
:1061C800626F727465642065646974730A00696E2D
:1061D80076616C69642073656C656374696F6E00C1
:1061E8000D0A496E76616C696420696E7075742059
:1061F8002D206469736361726465642107005365C7
:106208007474696E677320736176656420746F2097
:10621800454550524F4D0A00526576657274656463
:106228002073657474696E67732066726F6D20459C
:106238004550524F4D0A004C6F6164656420666199
:1062480063746F72792064656661756C74730A0093
:106258004B657920616E64206368616E6E656C734E
:106268002072616E646F6D697A65640A004F7065AB
:106278006E4C52536E67205458207374617274695F
:106288006E672000206F6E20485720006D6F647580
:106298006C65206C6F636B65643F00342B34003889
:1062A80000382B340031320031322B3400313600C3
:1062B80050504D0052535349005344410053434CEE
:1062C80000525844005458440041494E004C42453D
:1062D80045500053504B54524D00534255530053B0
:1062E800554D44004C4C494E440000070B0C10110E
:1062F8001500B7012B032F033103350338033D0382
:10630800B7014003440349034D035103550359039F
:106318005D0363036A036F0374038D028D028D02AC
:106328008D02160A1322312900000000C62BCB2942
:086338006C2B992B7E2BBB2B73
:00000001FF
